:020000040000FA
:040000000000B82A1A
:08000800F000030E83018312D6
:100010000313EF000A08EE008A011820831203136D
:100020006E088A0083016F0E8300F00E700E0900C7
:10003000831203130C1E452883160C1E45288312B9
:1000400003132B082A06031945282A08303EC0004E
:1000500001300318013EC100400884008313411899
:1000600083170008C200AA0A10302A020318AA0146
:100070002B082A06031D3F28831603130C12831234
:100080000313420883120313990083128C1E49281C
:10009000FF20831203130800831203132D08BC00F2
:1000A00008303C02031C58280830BC001030AD005A
:1000B000BD01831203138B1B602883120313BD0A37
:1000C000831203133D08031D6828831203138B1347
:1000D0005430DC20A90151302A22BE00DC2030300F
:1000E000BC043C082A22BC00DC202C082A22BC00CC
:1000F000DC208312031320082A22BC00DC20BC0170
:10010000831203132D083C02031898283C08403E34
:10011000BE0001300318013EBF003E088400831377
:100120003F18831700082A22BE00DC20BC0A802862
:10013000831203132908DC203D08031DA228831223
:1001400003138B1783120313080000308312031369
:100150002F04031DAD28BD22A52808008312031318
:100160002F08080000300800080083120313270836
:10017000BA20080083120313AC00AD0108008312FB
:100180000313AF01080083120313B90010302D02CE
:100190000318DB282D08BA00AD0A3A08403EBA0021
:1001A00001300318013EBB003A08840083133B185A
:1001B000831739088000080083120313B6002B0848
:1001C000303EB70001300318013EB8003708840004
:1001D000831338188317360880002B0AB6001030B6
:1001E00036020318B6012A0836060319F328360822
:1001F000AB00831603130C1683120313080083123B
:1002000003131A0883120313B30083120313981CF9
:100210000B2918120C291816831203132208B40094
:1002200030303402031C292A3B3034020318292AB7
:10023000D030B40701308A002330340703188A0A0B
:100240008312031382002E293729582982299A29DB
:10025000A429C229F5290E2A152A1D2A831203135F
:100260003308543A031D292A3130A200292A831267
:1002700003133308A400FC303305B400503A0319CB
:1002800048295430DC203308DC203730A200292AEA
:1002900003303305B400013A031D51290130B00089
:1002A0005229B001A90133082A223230A200292A9A
:1002B000831203133308A300F0303305B400303A3F
:1002C00003196B295430DC202408DC203308DC209F
:1002D0003830A200292A0F303305A500A51D7D293D
:1002E00007303305B4000830A5003408003C03197A
:1002F0007D29A50D013E031C792933082A223330BC
:10030000A200292A83120313200883120313330641
:10031000031995295430DC202408DC202308DC2034
:100320003308DC203930A200292A33082A2234304D
:10033000A200292A831203133308A600A801330858
:100340002A223530A200292A00302F04031DB829A3
:10035000831203132808203EB40001300318013E25
:10036000B5003408840083133518831733088000E0
:10037000A80A33082A2225082806031D292A363010
:10038000A200292A8312031329083306031DD52945
:100390002F080319CE295330B400D7295230B400A6
:1003A0000130AF002608A700D7295330B400003031
:1003B00030040319F2295430DC20A90134082A2220
:1003C000B400DC2030302A22B400DC2026082A22A7
:1003D000B400DC208312031320082A22B400DC209E
:1003E0002908DC203030A200292A831203133308A5
:1003F000DC200F303305A500A51D0B2A073033057F
:10040000B4000830A5003408003C03190B2AA50DE0
:10041000013E031C072A3830A200292A8312031345
:100420003308DC203930A200292A83120313330851
:10043000DC20A50A3A30A200292A831203133308CC
:10044000DC2002302502031C272AA503292A30308C
:10045000A200080083120313B1002906B200A9010B
:10046000321C342A5E30A906B21C382ABC30A906D8
:10047000321D3C2A6130A906B21D402AC230A906AD
:10048000321E442A9D30A906B21E482A2330A906EE
:10049000321F4C2A4630A906B21F502A8C30A906BA
:1004A00031080800303083120313A200AB01AA0107
:1004B000AF01080083120317200883120313A10061
:1004C000033021020318882A02308A006D30210788
:1004D00003188A0A831203138200702A792A802A59
:1004E000B5200030C3200030C3200130C3204C2091
:1004F000882A831203172108831203138600882A8F
:10050000B5200230C320831203130508C3204C20FA
:10051000080008009422892252220030DC20A52005
:100520005A22BF208F2A0800DF3083160313810070
:10053000FF3083129F00FF3083168500063086004F
:100540008C0183128B018C010C30831699000430CE
:10055000980080308312980083168C168312181628
:100560008316981683120B178B17860185010800D6
:0E057000323083120313A0008A2A64000800B0
:02400E00103F61
:00000001FF
